:1000000001308A0037290000D308031D1D28081776
:10001000881208128811081C132808180D28D50109
:100020002A30F8008428081D1B2808191528D50136
:100030002330F800842807288428530B8428881547
:10004000081388120812081C2A280818252831309D
:10005000F8008428881C312888182C283230F800B1
:100060008428081D3828081933283330F8008428DC
:100070000816081388128811081C432808183E28FF
:100080003430F8008428881C4A28881845283530E0
:10009000F8008428081D512808194C283630F8002B
:1000A00084288816081308128811081C5C28081870
:1000B00057283730F8008428881C632888185E2861
:1000C0003830F8008428081D6A2808196528393056
:1000D000F80084280817881208128811081C75284F
:1000E000081870282A30F8008428881C7C28881872
:1000F00077283030F8008428081D832808197E28C6
:100100002330F80084281F288A110A12B4295A3093
:1001100084008313000803199A280630F800F701B9
:10012000F70B9028F80B8F287B30F700F70B9628F9
:10013000800B8D28080058088600591C0710591894
:10014000071487140A30DA00872087100A30DA0093
:10015000872008005508033C03183429D5015508A9
:10016000D300D8012730D700DA012230D90058084F
:10017000FA005708840083137A1883170008DB00FD
:100180005A08FA005908840083137A188317000864
:100190005B02031DE2285808FA0057088400831305
:1001A0007A1883178008031DD8280030F800FA2831
:1001B0005808FA005708D70A0319D80AD90A0319A8
:1001C000DA0AB7285808FA00570884008313581829
:1001D00083170008DB005A08FA00590884008313CB
:1001E0005A18831700085B020318F828FF30F92813
:1001F0000130F8007808D600D608031D1A29071523
:100200000130D800D9019B208030D800D9019B2033
:10021000D4015408063C031C19293B3054078400C0
:1002200083130008D700D8000130D9009B20D40ADE
:100230000929342907110130D800D9019B208030C9
:10024000D800D9019B20D40154080D3C031C34294B
:1002500043305407840083130008D700D8000130CE
:10026000D9009B20D40A24298A110A12FF290308E5
:100270001F39830083161F149F141F159F11073009
:100280009C0083138312A001A1013730A2003130FA
:10029000A3003930A4003630A500A6014530AC00DB
:1002A0006E30AD007430AE006530AF007230B0001B
:1002B0002030B1005030B2006130B3007330B40070
:1002C000B5007730B6006F30B7007230B8006430D8
:1002D000B900BA015730BB006530BC006C30BD00BE
:1002E0006330BE006F30BF006D30C0006530C100AC
:1002F000C2015730C3007230C4006F30C5006E3089
:10030000C6006730C7002030C8005030C9006130D7
:10031000CA007330CB00CC007730CD006F30CE00F8
:100320007230CF006430D000D10183160711051060
:100330000710871086018811081288128312D501D0
:10034000831608138312551CA829831608178312D5
:100350008316081B8816881A0816081A88150815A7
:1003600088140814831204287808D20052082A3C02
:10037000031DE2290130D300D501D800D9019B200B
:100380003830D800D9019B200F30D800D9019B20EC
:100390008030D800D9019B20D40154080D3C031CA7
:1003A000DD292C305407840083130008D700D800BF
:1003B0000130D9009B20D40ACD29C030D800D90102
:1003C0009B20FF295208233C031DF129D501071169
:1003D0000130D800D9019B200C30D800D9019B20D6
:1003E000FF292A30D8000130D9009B20273055073B
:1003F00084008313520880000130D507AA28B3294E
:02040000630097
:02400E00323F3F
:00000001FF
